:1000000000308A005F280000FF00030E8301A1007A
:100010007F08A0000A08A8008A01A00E0408A20018
:100020007708A3007808A4007908A5007A08A6003C
:100030007B08A700831383128C308400801D222844
:100040008C193528220884002308F7002408F800BA
:100050002508F9002608FA002708FB0028088A006E
:10006000210E8300FF0E7F0E09008A1143280A101B
:100070008A100A118207023406340E341E343E34CC
:100080007E34FE34FF34290893008C118A11222813
:100090002F308400000803195E280130F800BF30BB
:1000A000F7006400F70B5128F80B4F284A30F7008F
:1000B000F70B582800006400800B4D2800348401A1
:1000C0001F30830583161F129F121B0880399B0067
:1000D00007309C001C0883120D13603083168F00BC
:1000E0000108C03981000E30F7000730831281010A
:1000F000813084000008F03907388000640000086F
:10010000F739F719F0397704800083161F129F1210
:100110001B088039D2389B001F1383121F179F17AB
:1001200083169F1383121F149412831606118614CC
:1001300006120030831294008316940083129001FB
:10014000073083169C00050864000230F700F70BA7
:10015000A728000000001C0883120D1383169D01C0
:1001600086118312861183160611831206118316D7
:100170008610831286102030F8001F08C7397804D3
:100180009F00950183168611831286110C3097000B
:100190000030F80004389200643083169200623018
:1001A0008F0002308312950083168610831286100A
:1001B0006430AF00482083168610831286141430F2
:1001C000AF0048201F151F19E3281E08783C031CA8
:1001D000D42883168610831286100830F8001F0872
:1001E000C73978049F0064002030F700F70BF62829
:1001F000000000001F151F19FB281E08F700031040
:10020000F70C7708283EAC0095010030F800043860
:1002100092002C088316920014308312950032301D
:10022000AE00FA30AF004820AE0B112983169401BE
:100230002230831294000230A90029089300C030B4
:100240008B0483168C158312AA012A08073C031C11
:1002500032292A083720F800A9003730AF0048209B
:10026000AA0A2529831694018312940183168C11FE
:100270000611831206150A30AE008230AF00482006
:10028000AE0B3D2983160611831206114629630021
:04400E003C2FFC3F08
:00000001FF
